:1000000012C0C9C02BC02AC029C028C027C026C022
:10001000A8C032C123C022C021C020C01FC01EC042
:100020001DC01CC01BC011241FBECFE5D4E0DEBF25
:10003000CDBF11E0A0E6B0E0E4E9F4E102C0059034
:100040000D92AA36B107D9F711E0AAE6B1E001C0D6
:100050001D92A237B107E1F71FD11ACAD1CFDF93A2
:10006000CF93CDB7DEB787E390E02FEFFC0120837D
:1000700088E390E0FC01108284E390E02FEFFC0124
:10008000208385E390E0FC01108281E390E020E38F
:10009000FC01208382E390E0FC011082CF91DF918C
:1000A0000895DF93CF93CDB7DEB782E390E022E3EC
:1000B00030E0F90120812061FC012083CF91DF91A4
:1000C0000895DF93CF93CDB7DEB782E390E022E3CC
:1000D00030E0F90120812F7EFC012083CF91DF9158
:1000E0000895DF93CF93CDB7DEB785E390E025E3A6
:1000F00030E0F90120812062FC012083CF91DF9163
:100100000895DF93CF93CDB7DEB785E390E025E385
:1001100030E0F90120812F7DFC012083CF91DF9118
:100120000895DF93CF93CDB7DEB785E390E025E365
:1001300030E0F90120812860FC012083CF91DF911C
:100140000895DF93CF93CDB7DEB785E390E025E345
:1001500030E0F9012081277FFC012083CF91DF91DE
:1001600008951F920F920FB60F9211248F939F93B1
:10017000DF93CF93CDB7DEB780EA9FE090936C0119
:1001800080936B01CF91DF919F918F910F900FBE64
:100190000F901F9018951F920F920FB60F92112477
:1001A0002F938F939F93EF93FF93DF93CF9300D081
:1001B000CDB7DEB780E390E0FC018081882F90E02E
:1001C00084709070009779F08EE490E0FC011082CA
:1001D0008CE490E0FC01118210828EE490E021E03A
:1001E000FC0120833BC080E390E0FC018081882FEC
:1001F00090E084709070009789F58EE490E0FC01A7
:1002000010828CE490E0FC01808191819A83898343
:1002100089819A81FDE781309F0738F088EE93E06D
:1002200090936C0180936B0119C089819A812EE3B0
:100230008038920728F410926C0110926B010EC066
:1002400089819A8180589E43929582958F708927E3
:100250009F70892790936C0180936B010F900F9092
:10026000CF91DF91FF91EF919F918F912F910F90FF
:100270000FBE0F901F9018951F920F920FB60F92FE
:100280001124DF93CF93CDB7DEB7CF91DF910F90DD
:100290000FBE0F901F9018950F931F93DF93CF936E
:1002A000CDB7DEB7AA970FB6F894DEBF0FBECDBFAD
:1002B000D6DE85E590E021E0FC0120838BE590E02F
:1002C00020E4FC0120838FE490E0FC01108289E5AA
:1002D00090E029E530E0F90120812460FC012083D1
:1002E0008EE490E0FC0110828CE490E0FC0111822D
:1002F000108283E590E021E0FC01208389E590E015
:1003000029E530E0F90120812160FC012083789407
:100310008EE490E021E0FC012083D3DEF2DE11DFE9
:1003200001C0000080916B0190916C01893C9105A6
:1003300008F49EC180916B0190916C0123E030E044
:10034000B90148D89B01C901CC01A0E0B0E0BC01D3
:10035000CD01E3D5DC01CB0189839A83AB83BC83D8
:1003600069817A818B819C8120E030E04AE755E405
:100370000FD4DC01CB018D839E83AF83B88711E05E
:100380006D817E818F81988520E030E040E85FE3D9
:100390004AD588230CF010E0112329F081E090E089
:1003A0009A87898742C011E06D817E818F8198850F
:1003B00020E03FEF4FE757E4E0D418160CF010E0D0
:1003C000112351F169817A818B819C8120E030E099
:1003D00040E251E4DDD3DC01CB01BC01CD0116D2FA
:1003E000DC01CB019A87898712C080E991E09C8764
:1003F0008B878B859C858C01C8010197F1F78C0157
:100400001C870B8789859A8501979A8789878985B3
:100410009A85009751F716C06D817E818F819885EE
:10042000F5D1DC01CB019A87898789859A859E87DA
:100430008D878D859E858C01F8013197F1F78F01AD
:100440001E870D872EDE7DDE80916B0190916C0101
:1004500023E030E0B901BED79B01C901CC01A0E087
:10046000B0E0BC01CD0159D5DC01CB018F87988B61
:10047000A98BBA8B6F85788989899A8920E030E0C9
:100480004AE755E485D3DC01CB018B8B9C8BAD8B8C
:10049000BE8B11E06B897C898D899E8920E030E0DC
:1004A00040E85FE3C0D488230CF010E0112329F06A
:1004B00081E090E0988F8F8B42C011E06B897C893E
:1004C0008D899E8920E03FEF4FE757E456D41816F8
:1004D0000CF010E0112351F16F85788989899A8990
:1004E00020E030E040E251E453D3DC01CB01BC0119
:1004F000CD018CD1DC01CB01988F8F8B12C080E9AC
:1005000091E09A8F898F898D9A8D8C01C80101970E
:10051000F1F78C011A8F098F8F89988D0197988F29
:100520008F8B8F89988D009751F716C06B897C89C6
:100530008D899E896BD1DC01CB01988F8F8B8F8940
:10054000988D9C8F8B8F8B8D9C8D8C01F8013197B2
:10055000F1F78F011C8F0B8FB4DDC3DD80916B0130
:1005600090916C0123E030E0B90134D79B01C901BF
:10057000CC01A0E0B0E0BC01CD01CFD4DC01CB01C7
:100580008D8F9E8FAF8FB8A36D8D7E8D8F8D98A12F
:1005900020E030E04AE755E4FBD2DC01CB0189A33F
:1005A0009AA3ABA3BCA311E069A17AA18BA19CA1E2
:1005B00020E030E040E85FE336D488230CF010E020
:1005C000112329F081E090E09EA38DA342C011E0A9
:1005D00069A17AA18BA19CA120E03FEF4FE757E4EE
:1005E000CCD318160CF010E0112351F16D8D7E8DD7
:1005F0008F8D98A120E030E040E251E4C9D2DC01C7
:10060000CB01BC01CD0102D1DC01CB019EA38DA3A6
:1006100012C080E991E098A78FA38FA198A58C01C3
:10062000C8010197F1F78C0118A70FA38DA19EA116
:1006300001979EA38DA38DA19EA1009751F716C08F
:1006400069A17AA18BA19CA1E1D0DC01CB019EA381
:100650008DA38DA19EA19AA789A789A59AA58C0192
:10066000F8013197F1F78F011AA709A74ADD59DD83
:1006700080916B0190916C01893C910508F051CEFD
:1006800020DD3FDD5EDD4ECEDF93CF93CDB7DEB70D
:100690002C970FB6F894DEBF0FBECDBF98878F831F
:1006A00069874A873C872B878F819885892F99276F
:1006B00023E030E0B9018ED6898389858095482F63
:1006C00050E08A85282F30E0429FC001439F900D63
:1006D000529F900D11242FEF30E0B9018FD69B016E
:1006E000C9018D838D818A838F819885AC0150707B
:1006F0008985282F30E0429FC001439F900D529F73
:10070000900D11242FEF30E0B90164D69B0189854B
:100710008095882F90E0A901480F591F8A85282FBE
:1007200030E0429FC001439F900D529F900D1124D5
:100730002FEF30E0B9014ED69B01C9018E838E8127
:100740008B838F81988580959095AC0150708985B9
:10075000282F30E0429FC001439F900D529F900D83
:1007600011242FEF30E0B90135D69B0189858095A2
:10077000882F90E0A901480F591F8A85282F30E063
:10078000429FC001439F900D529F900D11242FEF67
:1007900030E0B9011FD69B01C9018C838981882F64
:1007A00090E002969E012E5F3F4F820F931FFC0147
:1007B00020818B859C85FC0120838B859C850196FF
:1007C0002981222F30E02F5F3F4FAE014E5F5F4FF8
:1007D000240F351FF9012081FC0120838B859C8526
:1007E00002962981222F30E0AE014E5F5F4F240F29
:1007F000351FF9012081FC0120832C960FB6F89457
:10080000DEBF0FBECDBFCF91DF910895EF92FF9273
:100810000F931F937B018C0120E030E040E05FE408
:10082000D7D287FD0FC0C801B70120E030E040E01B
:100830005FE483D123D39B01AC0120503040404082
:10084000504805C0C801B70119D39B01AC01B901DB
:10085000CA011F910F91FF90EF900895A0E0B0E0C2
:10086000E3E3F4E0E2C5FC01EA018081823008F4B0
:1008700038C1DB019C91923008F430C1843059F4C6
:10088000943009F02EC1918111968C91119798178F
:1008900009F021C126C1943009F420C19230B1F48D
:1008A000823009F01EC1CA01AF0128E0DA010D90C3
:1008B000AD01DC010D92CD012150C1F7DB01119694
:1008C0008C9111979181892389830AC1823009F41F
:1008D00005C1C280D380DB0112966D907C90139786
:1008E00024813581468157811496ED90FD900D91BC
:1008F0001C911797C601861997095C0197FF04C0E0
:10090000AA24BB24A81AB90AB0E2AB16B1040CF0B1
:1009100061C0181619066CF5370148010A2C04C08D
:1009200096948794779467940A94D2F781E090E044
:10093000A0E0B0E00A2C04C0880F991FAA1FBB1FBB
:100940000A94D2F70197A109B1098E219F21A02312
:10095000B123EE24FF248701E3940097A105B1059C
:1009600019F4EE24FF248701E628F728082919291D
:100970003CC00097D1F1CA0CDB1C39014A010A2C9A
:1009800004C096948794779467940A94D2F781E090
:1009900090E0A0E0B0E00A2C04C0880F991FAA1FC5
:1009A000BB1F0A94D2F70197A109B10982239323AF
:1009B000A423B52321E030E040E050E00097A105FA
:1009C000B10519F420E030E0A9012629372948298A
:1009D00059290BC06C147D0424F4EE24FF248701F4
:1009E00004C0630120E030E0A9018181FB01918115
:1009F000891709F445C0882349F0D801C701821B33
:100A0000930BA40BB50B9C01AD0104C02E193F093B
:100A1000400B510B57FD04C01982DB82CA820BC008
:100A200081E08983DB82CA8250954095309521957B
:100A30003F4F4F4F5F4F2C833D834E835F830DC0ED
:100A4000880F991FAA1FBB1F8C839D83AE83BF8312
:100A50008A819B8101979B838A838C819D81AE8152
:100A6000BF819C01AD0121503040404050402F3F9C
:100A7000EFEF3E07EFEF4E07EFE35E0708F30BC023
:100A80008983DB82CA822E0D3F1D401F511F2C839C
:100A90003D834E835F8383E088832C813D814E813B
:100AA0005F8157FF1DC0DA01C90181709070A0708D
:100AB000B0705695479537952795822B932BA42B8D
:100AC000B52B8C839D83AE83BF838A819B810196E6
:100AD0009B838A8305C0E2E6F0E003C0FB0101C00E
:100AE000FE01CF01CDB7DEB7EEE0BBC4A0E2B0E0BF
:100AF000EBE7F5E0A2C469837A838B839C832D8323
:100B00003E834F83588789E0E82EF12CEC0EFD1EC2
:100B1000CE010196B7019CD38E010F5E1F4FCE010F
:100B20000596B80195D3C701B801AE01475E5F4F86
:100B300095DEC1D2A096E6E09CC4A0E2B0E0E2EA75
:100B4000F5E07BC469837A838B839C832D833E830A
:100B50004F8358878E01075F1F4FCE010196B80162
:100B600077D391E1E92EF12CEC0EFD1ECE01059616
:100B7000B7016ED38A8991E089278A8BC801B701B2
:100B8000AE01475E5F4F6ADE96D2A096E6E071C482
:100B9000A0E2B0E0EDECF5E044C469837A838B8396
:100BA0009C832D833E834F835887CE010196BE01DF
:100BB000675F7F4F4DD3CE010596BE016F5E7F4FBD
:100BC00047D39985923078F089898230C0F094308B
:100BD00019F4823041F4CBC0843019F4923079F4A6
:100BE000C6C0923051F481E02A859A89291709F408
:100BF00080E08A87CE010996BCC0823051F481E042
:100C00002A859A89291709F480E08A8BCE014196BA
:100C1000B0C06D847E848F849888ED88FE880F89AB
:100C2000188DE0E2F0E080E090E0DC01AA24BB2433
:100C3000650120E030E0A901B301617070706115B9
:100C40007105D1F02E0D3F1D401F511F15012601CA
:100C5000280E391E4A1E5B1E81E090E0A0E0B0E045
:100C60002E153F054007510718F080E090E0DC01A9
:100C7000820D931DA41DB51DAA0CBB1CCC1CDD1C34
:100C800017FF09C061E0262E312C412C512CA228DF
:100C9000B328C428D528319749F0EE0CFF1C001F5B
:100CA000111F9694879477946794C6CF6B897C893B
:100CB000EB85FC856E0F7F1F6E5F7F4F7C8F6B8F88
:100CC00061E0EA857A89E71709F460E06A8F6B8D45
:100CD0007C8D10C0FC01E170F070309729F05695C2
:100CE0004795379527955068B695A7959795879519
:100CF0006F5F7F4FB7FDEECF0CC0880F991FAA1F03
:100D0000BB1F57FD8160220F331F441F551F6150C9
:100D100070408030E0E09E07E0E0AE07E0E4BE0710
:100D200060F36B8F7C8F6FE7E62EF12C012D112D78
:100D3000E822F9220A231B2360E4E616F1040105E8
:100D4000110561F487FD0AC02115310541055105E2
:100D500029F0805C9F4FAF4FBF4F80788D8F9E8F63
:100D6000AF8FB8A383E0898FCE01499602C082E697
:100D700090E0A1D1A096E2E170C3A8E1B0E0E2EC7E
:100D8000F6E05BC369837A838B839C832D833E83E8
:100D90004F8358878E01075F1F4FCE010196B80120
:100DA00057D281E1E82EF12CEC0EFD1ECE01059606
:100DB000B7014ED28985823038F08989823020F09F
:100DC000C801B701AED201C08FEF6896E6E051C30B
:100DD000A8E1B0E0EDEEF6E030C369837A838B835F
:100DE0009C832D833E834F8358878E01075F1F4F5F
:100DF000CE010196B8012CD281E1E82EF12CEC0E47
:100E0000FD1ECE010596B70123D28985823038F0C8
:100E10008989823020F0C801B70183D201C08FEFE9
:100E20006896E6E026C3A8E1B0E0E8E1F7E005C394
:100E300069837A838B839C832D833E834F8358877A
:100E40008E01075F1F4FCE010196B80101D281E1EB
:100E5000E82EF12CEC0EFD1ECE010596B701F8D15F
:100E60008985823038F08989823020F0C801B70145
:100E700058D201C081E06896E6E0FBC2ACE0B0E089
:100E8000E3E4F7E0DEC269837A838B839C83CE013F
:100E90000196BE016B5F7F4FDBD18D81823081F186
:100EA000823070F1843021F48E81882369F10AC088
:100EB0002F81388537FD24C06E812F3131053CF0FC
:100EC000662311F120E030E040E050E821C08EE1DF
:100ED00090E0821B930B29853A854B855C8504C085
:100EE00056954795379527958A95D2F7662381F0D1
:100EF00050954095309521953F4F4F4F5F4F08C01B
:100F000020E030E0A90104C02FEF3FEF4FEF5FE793
:100F1000B901CA012C96E2E0B0C2A8E0B0E0E2E973
:100F2000F7E089C27B018C011A8261157105810588
:100F3000910519F482E089835EC083E089838EE1A4
:100F4000C82ED12CDC82CB82ED82FE820F831887E3
:100F5000C801B70156D0FC013197F7FF3AC0AA2764
:100F6000BB27AE1BBF0B21E030E040E050E00A2E73
:100F700004C0220F331F441F551F0A94D2F721507B
:100F80003040404050402E213F214023512361E01A
:100F900070E080E090E0211531054105510519F41C
:100FA00060E070E0CB0104C016950795F794E794D4
:100FB000AA95D2F7E62AF72A082B192BED82FE8292
:100FC0000F8318878EE190E08E1B9F0B9C838B8391
:100FD00012C0309781F00E2E04C0EE0CFF1C001FD3
:100FE000111F0A94D2F7ED82FE820F831887CE1A62
:100FF000DF0ADC82CB82CE0101965DD02896E8E044
:1010000036C2AF92BF92CF92DF92EF92FF920F93D0
:101010001F937B018C0180E0E81680E0F80681E0F8
:10102000080780E0180758F4EFEFEE16F104010509
:10103000110509F090F480E090E0DC0117C0F0E0C9
:10104000EF16F0E0FF06F0E00F07F1E01F0750F4A5
:1010500080E190E0A0E0B0E009C088E090E0A0E08E
:10106000B0E004C088E190E0A0E0B0E020E230E031
:1010700040E050E0281B390B4A0B5B0B570168011D
:1010800004C0D694C794B794A7948A95D2F7D60192
:10109000C50186599F4FFC018081281B31094109F8
:1010A0005109C9011F910F91FF90EF90DF90CF90F0
:1010B000BF90AF900895EF92FF920F931F93CF933D
:1010C000DF93FC01248135814681578161818081D4
:1010D000823020F44061EFEFF0E0A3C0843009F4E7
:1010E0009BC0823009F492C021153105410551059C
:1010F00009F48FC00280F381E02D8FEFE238F8070A
:101100000CF05AC0C2E8DFEFCE1BDF0BCA31D105AD
:101110006CF579018A010C2E04C016950795F79499
:10112000E7940A94D2F781E090E0A0E0B0E00C2EC2
:1011300004C0880F991FAA1FBB1F0A94D2F70197FA
:10114000A109B10982239323A423B52321E030E030
:1011500040E050E00097A105B10519F420E030E02F
:10116000A9012E293F29402B512B03C020E030E05C
:10117000A901DA01C9018F779070A070B070803436
:101180009105A105B10539F427FF09C0205C3F4F47
:101190004F4F5F4F04C0215C3F4F4F4F5F4FE1E027
:1011A000F0E0203080E0380780E0480780E458070E
:1011B00028F5E0E0F0E022C0E038F1056CF5E158F8
:1011C000FF4FDA01C9018F779070A070B070803442
:1011D0009105A105B10539F427FF09C0205C3F4FF7
:1011E0004F4F5F4F04C0215C3F4F4F4F5F4F57FF42
:1011F00005C05695479537952795319687E05695C2
:101200004795379527958A95D1F70BC0E0E0F0E038
:1012100005C0E0E0F0E005C0EFEFF0E020E030E0F6
:10122000A9018E2F879588278795942F9F7767959B
:1012300066276795E695E22EA92FA82BFE2FF62BA1
:10124000622F732F8A2F9F2FCDB7DEB7E6E011C133
:10125000DC01FB012C9111963C91119712968C9117
:101260001297482F4F7750E0982F991F9927991F71
:1012700013966C911397862F880F892B90E0661F29
:101280006627661F6183009739F5211531054105F1
:10129000510511F482E029C082E89FEF9383828395
:1012A00067E0220F331F441F551F6A95D1F783E073
:1012B000808309C0220F331F441F551F82819381F1
:1012C000019793838283203080E0380780E04807CD
:1012D00080E4580778F320C08F3F910579F42115F9
:1012E00031054105510519F484E08083089544FFD8
:1012F00003C081E0808310C010820EC08F579040E1
:101300009383828383E0808387E0220F331F441F0F
:10131000551F8A95D1F750642483358346835783BC
:101320000895FC01DB019081923008F449C08C9152
:10133000823008F445C0943051F461818430B1F5B5
:1013400011962C91119730E0261B310941C0843051
:1013500021F0923041F48230B1F111968C911197C5
:101360008823A1F12DC06181823001F111968C9109
:1013700011976817D9F42281338112968D919C912F
:1013800013978217930794F028173907BCF024812C
:1013900035814681578114968D919D910D90BC9118
:1013A000A02D82179307A407B50718F4662341F010
:1013B0000DC0281739074A075B0728F4662331F068
:1013C00021E030E005C020E030E002C02FEF3FEF29
:1013D000C9010895AA1BBB1B51E107C0AA1FBB1F6F
:1013E000A617B70710F0A61BB70B881F991F5A95B1
:1013F000A9F780959095BC01CD01089597FB092E22
:1014000007260AD077FD04D0E5DF06D000201AF4C5
:10141000709561957F4F0895F6F7909581959F4F50
:1014200008952F923F924F925F926F927F928F9288
:101430009F92AF92BF92CF92DF92EF92FF920F9363
:101440001F93CF93DF93CDB7DEB7CA1BDB0B0FB66D
:10145000F894DEBF0FBECDBF09942A88398848882A
:101460005F846E847D848C849B84AA84B984C884C0
:10147000DF80EE80FD800C811B81AA81B981CE0FB7
:10148000D11D0FB6F894DEBF0FBECDBFED0108959C
:04149000F894FFCFFE
:10149400010000000000000000000001020203033C
:1014A40003030404040404040404050505050505F4
:1014B40005050505050505050505060606060606D2
:1014C40006060606060606060606060606060606B8
:1014D40006060606060606060606070707070707A2
:1014E4000707070707070707070707070707070788
:1014F4000707070707070707070707070707070778
:101504000707070707070707070707070707070767
:101514000707070707070707070708080808080851
:101524000808080808080808080808080808080837
:101534000808080808080808080808080808080827
:101544000808080808080808080808080808080817
:101554000808080808080808080808080808080807
:1015640008080808080808080808080808080808F7
:1015740008080808080808080808080808080808E7
:1015840008080808080808080808080808080808D7
:0A15940008080808080808080808FD
:00000001FF
